:10000000082AA501A400B3172730A300103014203C
:100010000330A300E8301420A30164301420A301AE
:100020000A30142024081F28A2002508A100240853
:10003000A000C6212008031DB313B31B0800303EE7
:1000400022280408A2008316861283120930A30016
:1000500003103120A20CA30B292803143120031410
:10006000032A0318362800008612382886163828F6
:100070000030A10062306529083033190130A30037
:10008000A201360884003408362134088004032293
:10009000032284130005FF3E331DA20C3319A20D69
:1000A00032306421A30B432822080314032AA20040
:1000B000083033190130A300A20C3608840034083C
:1000C0003621340803188004373064213408800452
:1000D000A30B5C280314032AB31C032A7228B30061
:1000E000331C032A36088400340836210130A1006D
:1000F000E0306521340880040130A100E03065293A
:10010000B4003921200821040319032AF82184139B
:100110003408800664008C288D28A00A0319A10FDA
:100120008A288006032A3708A0003508A10001307C
:10013000A200A3016400BB20031CAE28A20B9A28D6
:10014000FF30A30703189A28A007031CA107031C6C
:1001500008006430A2000030A3009A28C6200830AE
:10016000A300C720BB20A20CB528A30BB128C72031
:100170000314220808003608840034088417800419
:100180008413000533193406FF3E0800331700308E
:100190008A00330D0639A000D920A10000308A0062
:1001A000200AD920331F65293313A000023085218E
:1001B0006529DD3E03188A0A820001348B3403343A
:1001C0002B34003452340C34EF34A40029080319C2
:1001D000032AFE21A0002518831724088400200884
:1001E00080008313A40AA903E628B313290803197E
:1001F000B3170430A800250E022125080221240E81
:10020000022124080F39F63E0318073E0A3E25292D
:10021000B31329080319B3170530A8002730A3002A
:1002200010301E210330A300E8301E21A3016430EA
:100230001E21A3010A301E2124082529A200250819
:10024000A1002408A000C6212008A000A8030319CB
:10025000B313290803192F292802031808002008BE
:10026000031DB313B31B0800303EFE29FF3A80057F
:100270003A29FF3A84178005032A031783168C0155
:100280000C1483120C0803178D0A032A03010317A9
:100290008C0083168C010C1555308D00AA308D0012
:1002A0008C148C1851290C1183128D0A032AA30176
:1002B000A200FF30A207031CA307031C032A03307C
:1002C000A100E33065215929A101F43EA000A10954
:1002D000FE30031C6E29A00703186B29A0076400D9
:1002E000A10F6B2900002018752920187729080014
:1002F000013EA7000A30A200A301C621A70B7D2959
:10030000240808000310A10CA00CFF3E031882294A
:100310002008032AA20002309D29A101A301A20006
:1003200003309D29A101A301A20001309D29A20053
:1003300006309D29A20004309D29A800230821022F
:10034000031DA429220820020430031801300319D8
:1003500002302805031DFF30032A0038031DFF303B
:100360000405031DFF30032A0404031DFF30032A84
:10037000A2002008A6002408A0002608A400210846
:10038000A6002508A1002608A500C829A501A401EA
:100390001030A600210DA40DA50D2208A4022308EB
:1003A000031C230FA5020318DC292208A407230835
:1003B0000318230FA5070310A00DA10DA60BCA2932
:1003C0002008032A1030A800A101A001A70CA60C48
:1003D000031CF0292208A00723080318230FA107F4
:1003E000A10CA00CA50CA40CA80BE6292408032A38
:1003F000A009A109A00A0319A10A08008400310874
:100400008A003008820083130313831264000800FB
:10041000C0309F00831671308F008312031787014D
:1004200088010313393090008316FF308500860160
:100430009F30870003170F30880089018312031350
:1004400041309F00831680309F00831286168316EA
:10045000861283120317F3308D0003138A013D21A6
:10046000F4000317FC308D0003138A013D21D200F4
:100470000317FD308D0003138A013D21D3000317BC
:10048000FE308D0003138A013D21E2000317FF3087
:100490008D0003138A013D21E3000317FA308D001C
:1004A00003138A013D21C8000317FB308D0003139D
:1004B0008A013D21C9000317F8308D0003138A011A
:1004C0003D21DA000317F9308D0003138A013D2125
:1004D000DB000317F4308D00031352088A01472113
:1004E0000317F5308D00031353088A0147210317C2
:1004F000F6308D0003135A088A0147210317F7309D
:100500008D0003135B088A0147210330A300E83004
:100510008A0158210614831606101B3083128A01A3
:10052000222046308A0122201B308A0122202E30D0
:100530008A0122201B308A01222043308A01222096
:1005400042308A0122204D308A01222053308A0114
:10055000222020308A0122204D308A012220613061
:100560008A01222073308A01222074308A012220DD
:1005700065308A01222072308A01222020308A01CF
:10058000222056308A01222030308A0122202E304B
:100590008A01222031308A01222036308A0122202D
:1005A00042308A01222079308A01222020308A01BB
:1005B000222050308A01222065308A0122207430A6
:1005C0008A01222065308A01222072308A0122208D
:1005D00020308A01222050308A01222065308A0191
:1005E000222072308A0122206B308A012220693059
:1005F0008A0122206E308A01222073308A01222053
:1006000077308A01222077308A01222077308A01D0
:1006100022202E308A01222031308A0122203530DA
:100620008A01222030308A0122206D308A01222066
:1006300070308A01222067308A0122202E308A0100
:10064000222063308A0122206F308A0122202E303E
:100650008A01222075308A0122206B308A012220F3
:100660000A308A0122200D308A01222038308A0186
:1006700022206D308A01222068308A0122207A30BF
:100680008A01222020308A01222028308A0122205B
:1006900001308A01012029308A01222020308A017C
:1006A000222043308A01222065308A0122206C30CA
:1006B0008A0122206C308A01222073308A01222094
:1006C00021308A0122200730A300D0308A0158212E
:1006D0000610831606101B3083128A012220433035
:1006E0008A012220DB30D6000B30D70056088E005E
:1006F00057088F000C100830860683168611831267
:100700008A110A122D248A150A12FE208A150A124D
:10071000B9228A150A1203266908A100043C8A112D
:100720000A12031CB62BA10D8A110A12A523A000E0
:1007300021108A110A12A5238A110A12A2238A11F2
:100740000A12B62B8A002008820003308A00210892
:10075000AC3E03188A0A82000E345F340E344C34E7
:100760000E3427340E3438340E34873464000130AC
:1007700070028A110A12031CC12BF10A8A110A1293
:10078000C22BF1017108A00002308A018D21DC002A
:100790007008A00000308A019221DE005C0884000D
:1007A0005E088A01AD21DE00DF0064005E085F04A0
:1007B0008A110A120319DF2B8A150A123024F0015C
:1007C000FB0A64007B08283C8A110A12031D212CB5
:1007D0000317FC308D00031352088A0147210317C9
:1007E000FD308D00031353088A0147210317FE30A3
:1007F0008D00031362088A0147210317FF308D0023
:10080000031363088A0147210317FA308D0003138D
:1008100048088A0147210317FB308D00031349085C
:100820008A0147210317F8308D0003135A088A0103
:1008300047210317F9308D0003135B088A01472114
:10084000FB0164008A110A120C1C212C56088E0030
:1008500057088F000C108A017B2B06158316061192
:10086000033083128A0157210611831606110130C5
:1008700083128A0157212830A000A101063084008C
:1008800004308A018020FF30E600E701D401D50161
:1008900032308A0157210615831606110330831260
:1008A0008A015721061183160611013083128A012D
:1008B00057211430A000A1010630840004308A01C1
:1008C00080200130E4006400023064028A110A12C0
:1008D0000318BC2CC201C30164007408003C8A11D7
:1008E0000A12031D762C8A110A12762C6400420823
:1008F00067028A110A120318812C4208E700640873
:10090000F8006400660842028A110A1203188C2C4F
:100910004208E6006408F900AF30C2070318C30AB2
:100920004208A0004308A1000130A3007C308A01E6
:1009300097218A110A12031DA12C0130F0006408CE
:10094000F7004208A0004308A100A301DC308A019F
:100950008F218A110A12031DB12C0230F0006408A5
:10096000F7004208D40743080318013ED507E40AFC
:100970008A110A12031D632C061583160611033013
:1009800083128A0157210611831606110130831242
:100990008A0157213C30A000A101063084000430B8
:1009A0008A01802064007508013C8A110A12031D27
:1009B000012D5408A0005508A1004F08A3004E08BF
:1009C0008A018F218A110A12031DFD2C5408CE02C0
:1009D0005508031C013ECF024E08A0004F08A1009D
:1009E000A30132308A0197218A110A12031DFA2CC1
:1009F0000630F0008A110A12012D5408CE00550865
:100A0000CF005408A0005508A1006430A200A30143
:100A10008A01C621E4002108E5005408A000550819
:100A2000A1006430A200A3018A01C6212408DC00D1
:100A30002508DD005C08A0005D08A1000A30A200C6
:100A4000A3018A01C621E8002108E9006408831691
:100A5000A0001B3083128A01222053308A012220F9
:100A600000308A01222000308A01222056308A017B
:100A700022206F308A0122206C308A01222020300F
:100A80008A0122206508A50064088A0102202E3010
:100A90008A0122206908A50068088A010220203006
:100AA0008A01222056308A01222020308A01222009
:100AB000AF306707E400E501E50D6408A0006508B4
:100AC000A1000130A3006D308A0197218A110A121A
:100AD000031D752D8614831686108312071783163F
:100AE000071383128A110A12792D0713831607132D
:100AF00083126408A0006508A1006430A200A3016D
:100B00008A01C621E8002108E9006408A000650800
:100B1000A1006430A200A3018A01C6212408EA00D2
:100B20002508EB007808E4001B308A0122205330AE
:100B30008A01222000308A01222001308A012220ED
:100B400048308A01222069308A01222056308A01E9
:100B5000222020308A0122205B308A01222064007A
:100B60000A3064028A110A120318B92D30308A0142
:100B700022206A08A0006B08A100A3010A308A01A4
:100B80008F218A110A12031DEA2D64088A010120AF
:100B90005D308A01222020308A0122206908A500C8
:100BA00068088A0102202E308A01222030308A0112
:100BB00022206B08A5006A088A01022020308A01E1
:100BC000222056308A01222020308A0122208A11D8
:100BD0000A12092E64088A0101205D308A01222050
:100BE00020308A0122206908A50068088A010220B5
:100BF0002E308A0122206B08A5006A088A01022093
:100C000020308A01222056308A01222020308A0199
:100C10002220AF306607E400E501E50D6408A0007E
:100C20006508A100A301E6308A018F218A110A120A
:100C3000031D252E061683160612831287168316A9
:100C4000871283128A110A122D2E0612831606129B
:100C5000831287128316871283126408A000650826
:100C6000A1006430A200A3018A01C621E800210886
:100C7000E9006408A0006508A1006430A200A30197
:100C80008A01C6212408EA002508EB007908E4005F
:100C90001B308A01222053308A01222000308A0131
:100CA000222002308A0122204C308A0122206F301B
:100CB0008A01222056308A01222020308A012220F7
:100CC0005B308A01222064000A3064028A110A1211
:100CD00003186D2E30308A0122206A08A0006B08AC
:100CE000A100A3010A308A018F218A110A12031D73
:100CF0009E2E64088A0101205D308A012220203066
:100D00008A0122206908A50068088A0102202E3085
:100D10008A01222030308A0122206B08A5006A084F
:100D20008A01022020308A01222056308A012220A6
:100D300020308A0122208A110A12BD2E64088A01FD
:100D400001205D308A01222020308A01222069089A
:100D5000A50068088A0102202E308A0122206B0833
:100D6000A5006A088A01022020308A01222056301C
:100D70008A01222020308A01222008006408F7001E
:100D80000330F0000800E601E701E401E501493025
:100D90009F000130E90064000B3069028A110A12D9
:100DA0000318EB2E9F1464008A110A129F1CDA2E7E
:100DB0008A01D32E1E08EB0083161E088312EA0058
:100DC0006A08E4076B080318013EE507E90A8A117F
:100DD0000A12031DCB2E4D309F000130E900640044
:100DE0000B3069028A110A1203180F2F9F14640036
:100DF0008A110A129F1CFE2E8A01F72E1E08ED0092
:100E000083161E088312EC006C08E6076D080318B1
:100E1000013EE707E90A8A110A12031DEF2E660850
:100E2000A0006708A1000A30A200A3018A01C62120
:100E3000E6002108E7006408A0006508A1000A3068
:100E4000A200A3018A01C621E4002108E5001830B0
:100E50006402FD0018306602FE007D08A0002D30FF
:100E60008A019221DC007E08A0002D308A019221A7
:100E7000DE005C0884005E088A01B421DE00DF0029
:100E800064005E085F048A110A120319492F0430B6
:100E9000F0001B308A01222053308A0122200030CA
:100EA0008A01222003308A01222054308A01222024
:100EB00065308A0122206D308A01222020308A018B
:100EC000222046308A01222064088A010120203035
:100ED0008A01222052308A01222066088A010120DC
:100EE00020308A012220F8308A01222043308A01F2
:100EF000222020308A01222008001B308A01222073
:100F000053308A01222000308A01222003308A01D6
:100F1000222054308A01222065308A0122206D303F
:100F20008A01222020308A0122200730B6000430B6
:100F3000B40001308A016F2055308A0157202830D3
:100F40008A01572010308A01572046308A015720E5
:100F500016308A01572001308A01572000308A015B
:100F6000572000308A015720AA308A015720BE300E
:100F70008A0157208A016C208A150A12382007300E
:100F8000B6000430B40001308A016F2055308A0168
:100F9000572028308A01572010308A0157204630C8
:100FA0008A01572016308A01572001308A015720C4
:100FB00000308A01572000308A015720AA308A0168
:100FC000572044308A0157208A016C200730B60030
:100FD0000430B40001308A016F2055308A01572057
:100FE00028308A0157200E308A0157202D308A017F
:100FF0005720EA308A01572000308A0157200030FC
:101000008A01572000308A0157204B308A0157202F
:10101000BE308A0157208A016C208A150A123820B6
:101020000730B6000430B40001308A016F2055301B
:101030008A01572028308A0157200E308A01572014
:101040002D308A015720EA308A01572000308A016A
:10105000572000308A01572000308A0157204B303A
:101060008A01572044308A0157208A016C200800E9
:101070000730B6000430B40002308A016F208A01C4
:101080003C20D8008A013C20D9008A016C206400F1
:101090008A150A12D919A4282B30F3007130A60042
:1010A0000230A7005808A2005908A3008A01E221D3
:1010B000F600A3010A308A01B821E0002108E1000E
:1010C000F0305805DC000F305905DD005C08A00049
:1010D0005D08A10004308A018521E0002108E100BB
:1010E0000F305805DC00DD015C08A6005D08A70094
:1010F0007130A2000230A3008A01E221CC00250851
:10110000CD0073088A012220A9016008A4006108AB
:10111000A5002130B000B1018A0108212E308A01DA
:101120002220A9014C08A4004D08A5002130B000E0
:10113000B1018A010821DF308A01222020308A0192
:1011400022208A150A12FD282D30F3005809DC00F0
:101150005909DD007130A6000230A7005C08A2002A
:101160005D08A3008A01E221DC002508DD005C0A9D
:10117000F600A3010A308A01B821E0002108E1004D
:1011800073088A012220A9016008A0006108A1005B
:1011900004308A017821DC00DD015C08A4005D08D0
:1011A000A5002130B000B1018A010821A901600821
:1011B000A0006108A10003308A017821DC00DD0174
:1011C0005C08A4005D08A5002130B000B1018A01CF
:1011D00008212E308A0122200330A9006008A400D3
:1011E0006108A5002130B000B1018A010821DF307B
:1011F0008A01222020308A0122200800E601E7012E
:1012000041309F000130E50064000B3065028A1513
:101210000A12031825299F1464008A150A129F1CBC
:1012200014298A150A120C291E08C10083161E08EB
:101230008312C0004008E60741080318013EE70793
:10124000E50A8A150A12031D04296608A00067082A
:10125000A1000A30A200A3018A01C621C000210812
:10126000C1004008A0004108A1000130A300FB30EC
:101270008A018F218A150A12031D57294008A000F0
:101280004108A1000330A200A3018A01C621DC00AD
:101290002108DD005C08FE3CC0005D08031C013E27
:1012A000013CC1002B30F3008A150A127329400853
:1012B000A0004108A1000230A30000308A0197215C
:1012C0008A150A12031D6F29AA30C0020030031CC0
:1012D000013EC1022D30F3008A150A127329C001A4
:1012E000C1013D30F3005408A0005508A10064304E
:1012F000A200A3018A01C621DC002108DD005C08F0
:10130000A6005D08A7004008A2004108A3008A01CA
:10131000E221E4002508E5006408A0006508A100BA
:10132000E830A2000330A3008A01C6212408DC00B3
:101330002508DD005C08A0005D08A1006430A20063
:10134000A3018A01C621E6002108E7006408A00085
:101350006508A100E830A2000330A3008A01C6217D
:10136000E4002108E5001B308A01222053308A0165
:10137000222000308A01222004308A0122204130BC
:101380008A0122206D308A01222070308A012220B9
:1013900020308A01222073088A0122204108A500FA
:1013A00040088A01022020308A0122204B308A0125
:1013B000222020308A0122206508A50064088A01C5
:1013C00002202E308A0122206708A50066088A01C3
:1013D000022020308A0122204008A6004108A700F0
:1013E0006430A200A3018A01E221DC002508DD00AF
:1013F0005C08A0005D08A1002430A200A3018A01BE
:10140000C621C0002108C100640073082B3C8A1566
:101410000A12031D292A4008C40741080318013E87
:10142000C5074408A0004508A100A30114308A01A3
:101430009A218A150A12031D292ADA0A0319DB0ADE
:101440001430C4020030031C013EC5028A150A1282
:10145000112A640073082D3C8A150A12031D512AB3
:101460004008C60741080318013EC7074608A00008
:101470004708A100A30114308A019A218A150A1293
:10148000031D512A0130DA020030031C013EDB0249
:101490001430C6020030031C013EC7028A150A122E
:1014A000362A5A08A0005B08A1006430A200A301FC
:1014B0008A01C621E8002108E9005A08A0005B085B
:1014C000A1006430A200A3018A01C6212408E4001F
:1014D0002508E5001B308A01222053308A01222092
:1014E00000308A01222005308A01222053308A01EF
:1014F00022206F308A01222063308A01222020308E
:101500008A0122206908A50068088A0102202E307D
:101510008A0122206408A0006508A100A3010A3006
:101520008A018F218A150A12031DAA2A30308A01E6
:1015300022206508A50064088A01022020308A0163
:10154000222025308A01222020308A0122208A157B
:101550000A12B82A6508A50064088A010220203012
:101560008A01222025308A01222020308A0122206F
:1015700008006608A0006708A100A30100308A01E6
:101580008A218A150A12031DE52A6608A000670849
:10159000A1000B30A200A3018A01C621E6002108A8
:1015A000E700E430A0001E30A1006608A200670832
:1015B000A3008A01C621DC002108DD0001305C07A0
:1015C000E6005D080318013EE7001B308A01222077
:1015D00053308A01222000308A01222006308A01FD
:1015E00022204D308A01222070308A01222068306A
:1015F0008A01222020308A0122206708A50066087F
:101600008A01022020308A01222077308A0122209C
:1016100068308A0122202F308A0122206D308A0111
:10162000222020308A0122206F08A5006E088A013E
:10163000022020308A01222020308A0122206608E0
:10164000A6006708A7009230A200A3018A01E22148
:10165000E6002508E7006608C80767080318013E8A
:10166000C9074808A0004908A100CE30A3004030B7
:101670008A019A218A150A12031DA82BFF0AE20A81
:101680000319E30A640064080A3C8A150A12031D60
:101690009F2BD20A0319D30A64085202E40065089A
:1016A000031C013E5302E5005A086802E6005B088D
:1016B000031C013E6902E7006608A0006708A1005C
:1016C0006408A2006508A3008A01C621E800210879
:1016D000E9005A08A0005B08A1006808A200690898
:1016E000A3008A01C621EA002108EB006A08CA00AB
:1016F0006B08CB006808A6006908A7000430A200A8
:10170000A3018A01E221DC002508DD005C08A600B7
:101710005D08A7001030A200A3018A01E221DC00CD
:101720002508DD005C08A0005D08A1006430A2006F
:10173000A3018A01C621EE002108EF00FF0140301D
:10174000C802CE30031C013EC9028A150A12312B91
:101750001B308A01222053308A01222000308A0166
:10176000222007308A0122204F308A012220643053
:101770008A0122206F308A01222020308A01222013
:101780005308A50052088A01022020308A01222035
:1017900052308A01222065308A0122206D308A0170
:1017A000222020308A0122204B08A5004A088A0105
:1017B000022020308A0122206208A0006308A100D4
:1017C0000A30A200A3018A01C621E4002108E50035
:1017D0006208A0006308A1000A30A200A3018A01E8
:1017E000C6212408E6002508E7001B308A012220D4
:1017F00053308A01222000308A01222008308A01D9
:10180000222054308A01222072308A01222069303D
:101810008A01222020308A0122206508A500640860
:101820008A0102202E308A0122206708A50066085E
:101830008A01022020308A01222043308A0122209E
:1018400068308A01222067308A01222020308A01F4
:10185000222075088A01012020308A0122200800F8
:101860001B308A0122205E308A01222064308A01E6
:1018700057211B308A01222021308A0122201B306F
:101880008A01222043308A01222020308A0122202E
:101890002A308A01222020308A01222042308A0107
:1018A00022204D308A01222053308A01222020300C
:1018B0008A01222041308A0122206C308A012220B4
:1018C00061308A01222072308A0122206D308A0123
:1018D000222073308A01222020308A0122202A30DF
:1018E0008A01222020308A0122200A308A01222007
:1018F0000D308A01222006148316061083128614E6
:101900008316861083120616831606128312061398
:10191000831606138312F50164007008013C8A15D2
:101920000A12031DBD2C43308A01222065308A0132
:1019300022206C308A0122206C308A012220203043
:101940008A01222077088A01012020308A01222082
:101950003E308A01222041308A0122204D308A0106
:10196000222061308A01222078308A0122205630DC
:101970008A01222020308A01222064007008023C63
:101980008A150A12031DEE2C43308A01222065308D
:101990008A0122206C308A0122206C308A012220A8
:1019A00020308A01222077088A01012020308A0114
:1019B00022203C308A01222041308A0122204D30F1
:1019C0008A01222069308A0122206E308A01222079
:1019D00056308A01222020308A01222064007008BB
:1019E000033C8A150A12031D1C2D43308A01222054
:1019F00065308A0122206C308A0122206C308A01F5
:101A0000222020308A01222077088A0101202030FC
:101A10008A01222045308A01222072308A01222048
:101A200072308A0122206F308A01222072308A01AE
:101A3000222021308A01222064007008043C8A158B
:101A40000A12031D532D50308A01222061308A0171
:101A5000222063308A0122206B308A0122203E300E
:101A60008A01222041308A01222062308A0122200C
:101A700073308A0122204D308A01222061308A0190
:101A8000222078308A01222054308A0122206530B9
:101A90008A0122206D308A01222070308A012220A2
:101AA00020308A01222064007008053C8A150A1241
:101AB000031D8A2D20308A01222020308A01222015
:101AC00041308A0122206C308A01222061308A0153
:101AD000222072308A0122206D308A01222020309B
:101AE0008A01222054308A01222065308A01222076
:101AF00073308A01222074308A01222021308A0129
:101B0000222020308A01222020308A012220203009
:101B10008A01222064007008063C8A150A12031DFF
:101B2000F12D20308A01222020308A0122204330EA
:101B30008A01222068308A01222061308A01222015
:101B400072308A01222067308A01222065308A01A2
:101B5000222020308A01222045308A0122206E3046
:101B60008A01222064308A01222021308A01222029
:101B700020308A01222020308A01222020308A0150
:101B8000222020308A01222056308A0122206F3004
:101B90008A0122206C308A01222074308A0122209E
:101BA00061308A01222067308A01222065308A0153
:101BB000222020308A01222044308A0122207230E3
:101BC0008A0122206F308A01222070308A0122206F
:101BD00020308A01222020308A01222020308A01F0
:101BE0002220F001F1010330A300E8308A015821DE
:101BF0000610831606101B3083128A0122205F30E4
:101C00008A012220080045309F009F1464008A1535
:101C10000A129F1C0E2E8A150A12062E1E08E900B3
:101C200083161E088312E8006808A0006908A10056
:101C30000430A200A3018A01C621DC002108DD00D6
:101C40000030DC070318DD0A5C03E9000800E2014C
:101C5000E3010317FE308D00031362088A01472158
:101C60000317FF308D00031363088A014721080022
:101C7000D201D3010317FC308D00031352088A01EF
:101C800047210317FD308D00031353088A014721B4
:101C900008000530F00008001030DA002730DB00C3
:101CA0000317F8308D0003135A088A0147210317E0
:101CB000F9308D0003135B088A0147210800640096
:101CC000013070028A150A12031C672E0800640096
:101CD0007508003C8A150A12031D812E0130F5009B
:101CE000861083168610831206128316061283123C
:101CF0000617831606138312CE01CF018A150A1226
:101D0000862EF501061383160613831208001B3076
:101D10008A0122205E308A01222064308A01572104
:101D20001B308A01222043308A0122202A308A0176
:101D3000222020308A01222020308A0122202030D7
:101D40008A01222053308A01222075308A01222004
:101D500062308A01222020308A0122204D308A01FF
:101D6000222065308A0122206E308A0122207530BF
:101D70008A01222020308A01222020308A0122205C
:101D800020308A0122202A308A0122200A308A014A
:101D900022200D308A01222043308A012220653022
:101DA0008A0122206C308A0122206C308A01222094
:101DB00020308A01222056308A0122206F308A0189
:101DC00022206C308A01222074308A012220613066
:101DD0008A01222067308A01222065308A01222070
:101DE00020308A0122203D308A01222020308A01C1
:101DF000222055308A01222053308A0122206C3063
:101E00008A01222061308A01222076308A01222034
:101E100065308A01222020308A01222055308A0133
:101E2000222070308A01222064308A012220613011
:101E30008A01222074308A01222065308A01222002
:101E400020308A0122203D308A01222020308A0160
:101E500022204C308A01222054308A0122207830FE
:101E60008A01222020308A01222042308A01222049
:101E70004D308A01222053308A01222020308A01ED
:101E8000222044308A01222061308A0122207430CD
:101E90008A01222061308A01222020308A012220FA
:101EA00020308A0122203D308A01222020308A0100
:101EB000222044308A01222054308A0122206530B9
:101EC0008A0122206D308A01222070308A0122206E
:101ED00020308A01222052308A0122206F308A016C
:101EE00022206D308A01222020308A0122202030D9
:101EF0008A01222020308A01222020308A012220DB
:101F000020308A0122203D308A01222020308A019F
:101F1000222052308A01222045308A012220783046
:101F20008A01222069308A01222074308A0122200D
:101F300020308A01222020308A01222020308A018C
:101F4000222020308A01222020308A0122202030C5
:101F50008A01222020308A01222020308A0122207A
:101F600020308A0122203D308A01222020308A013F
:101F7000222043308A0122200730A300D0308A017A
:101F800058218A150A12032664006908003C8A1148
:101F90000A1603194A2864006908013C8A110A16C6
:101FA0000319322964006908023C8A150A120319D0
:101FB000EE2F64006908043C8A150A120319E32F06
:101FC0008A150A12C12F1B308A0122205F308A0134
:101FD0002220080005308A01572108001B308A01A1
:101FE000222043308A01222053308A01222065308A
:101FF0008A0122206E308A01222064308A01222048
:1020000069308A0122206E308A01222067308A01DD
:10201000222020308A0122205108A50050088A0180
:1020200002200A308A0122200D308A01222042300B
:102030008A01222079308A01222074308A012220EC
:1020400065308A01222073308A01222020308A01E3
:10205000222042308A01222065308A01222020304D
:102060008A01222050308A01222061308A012220F8
:1020700074308A01222069308A01222065308A0169
:1020800022206E308A01222074308A0122208A1593
:102090000A12E32F1B308A01222043308A012220BA
:1020A0000130E5006400023065028A110A16031847
:1020B000E128C201C3016808A0006908A100A301CA
:1020C0000A308A018F218A110A16031D9E28433087
:1020D0008A01222065308A0122206C308A01222068
:1020E0006C308A01222020308A01222065088A0172
:1020F000012020308A01222020308A012220670816
:10210000A50066088A0102202E308A012220303084
:102110008A0122206908A50068088A010220563039
:102120008A01222020308A0122200A308A012220BE
:102130000D308A0122208A110A16CF2843308A01E5
:10214000222065308A0122206C308A0122206C30E6
:102150008A01222020308A01222065088A0101207C
:1021600020308A01222020308A0122206708A50021
:1021700066088A0102202E308A0122206908A50003
:1021800068088A01022056308A01222020308A0104
:1021900022200A308A0122200D308A0122207D303F
:1021A0008A0157218A150A12032664006908013C36
:1021B0008A110A16031DD228E50A8A110A16031D80
:1021C00052280130A300F4308A0158210A308A01D4
:1021D00022200D308A01222041308A0122206E30D7
:1021E0008A01222079308A01222020308A0122208F
:1021F0004B308A01222065308A01222079308A0101
:10220000222020308A01222054308A0122206F307F
:102210008A01222020308A01222045308A01222092
:1022200078308A01222069308A01222074308A01A4
:10223000222021308A0122200330A300E8308A01C5
:1022400058218A150A12032664006908053C8A1180
:102250000A16031921291B308A0122205F308A01C6
:10226000222008000930E8001B308A012220433078
:102270008A0122202A308A01222020308A0122204D
:1022800053308A0122206C308A01222061308A0179
:10229000222076308A01222065308A0122202030D7
:1022A0008A01222055308A01222070308A012220A2
:1022B00064308A01222061308A01222074308A0130
:1022C000222065308A01222020308A0122202A30F3
:1022D0008A01222020308A01222055308A012220C2
:1022E00073308A01222065308A01222020308A0141
:1022F000222055308A01222070308A0122202F307E
:102300008A01222044308A0122206F308A01222053
:1023100077308A0122206E308A01222020308A0103
:10232000222074308A0122206F308A01222020303E
:102330008A01222020308A01222053308A01222063
:1023400065308A0122206C308A01222065308A01A2
:10235000222063308A01222074308A01222020301A
:102360008A01222043308A0122206F308A012220F4
:102370006D308A0122206D308A01222061308A016D
:1023800022206E308A01222064308A0122202030EF
:102390008A0122200A308A0122200D308A0122205F
:1023A00020308A01222043308A01222065308A01B0
:1023B00022206E308A01222074308A01222072305D
:1023C0008A01222065308A01222020308A012220C1
:1023D00050308A01222075308A01222073308A0110
:1023E000222068308A01222020308A012220743085
:1023F0008A0122206F308A01222020308A01222087
:1024000020308A01222053308A01222065308A013F
:1024100022206E308A01222064308A01222020305E
:102420008A01222043308A0122206F308A01222033
:102430006D308A0122206D308A01222061308A01AC
:1024400022206E308A01222064308A01222021302D
:102450008A01222021308A0122200330A300E830A3
:102460008A0158218A150A1203261B308A0122206C
:1024700053308A01222000308A01222007308A014D
:10248000222020308A01222043308A0122206F300E
:102490008A0122206D308A0122206D308A0122209B
:1024A00061308A0122206E308A01222064308A0144
:1024B000222020308A01222068088A010120203051
:1024C0008A01222021308A01222020308A01222004
:1024D0000130A300F4308A01582164006908053CEA
:1024E0008A110A160319322A64006908003C8A110D
:1024F0000A16031D7C2AE80A64006908023C8A1156
:102500000A16031D842AE80364006908043C8A1142
:102510000A16031D322A0A308A0122200D308A0150
:10252000222043308A0122206F308A0122206E301F
:102530008A01222066308A01222069308A01222005
:1025400072308A0122206D308A01222020308A01D7
:10255000222020308A01222028308A01222059306E
:102560008A0122202F308A0122204E308A01222027
:1025700029308A01222020308A0122203F308A011E
:10258000222055308A01222070308A0122203D30DD
:102590008A01222059308A01222065308A012220B6
:1025A00073308A01222020308A01222044308A019F
:1025B00022206F308A01222077308A0122206E305B
:1025C0008A0122203D308A0122204E308A012220B9
:1025D0006F308A01222020308A01222021308A0196
:1025E00022200730A300D0308A0158218A150A1210
:1025F000032664006908003C8A110A1603190A2B95
:1026000064006908023C8A110A1603192D2C8A11EC
:102610000A16F62A1B308A01222043308A01222022
:1026200020308A01222043308A0122206F308A0123
:1026300022206D308A0122206D308A0122206130F3
:102640008A0122206E308A01222064308A012220F1
:1026500020308A01222068088A01012020308A0166
:10266000222053308A01222065308A0122206E30D8
:102670008A01222074308A01222021308A012220FE
:102680006808A600A7011430A200A3018A01E22174
:10269000EA002508EB00640068080A3C8A110A1663
:1026A000031D532BF401640068080B3C8A110A16C1
:1026B000031D5C2B0130F400061583160611033050
:1026C00083128A01572106118316061101308312E5
:1026D0008A0157216A08A0006B08A1000630840017
:1026E00004308A0180200130E4006400023064027A
:1026F0008A110A160318F22B64007408003C8A1130
:102700000A16031D962B0730B6008030B400063041
:10271000B3003230B700B5018A0193208A110A163E
:10272000031C742CE9008A110A16A62B0730B60088
:102730008030B4000430B3003230B700B5018A01F4
:1027400093208A110A16031C742CE900640068089F
:1027500069028A110A160319ED2B0A308A01222018
:102760000D308A01222053308A0122206C308A01E8
:10277000222061308A01222076308A0122206530B1
:102780008A01222020308A01222064088A01012047
:1027900020308A01222045308A01222072308A01AD
:1027A000222072308A0122206F308A01222072306A
:1027B0008A01222021308A01222006148316061065
:1027C00083120B30A300B8308A01582106108316FB
:1027D000061083128A110A162D2CE40A8A110A1691
:1027E000031D752B0A308A0122200D308A01222018
:1027F00041308A01222063308A0122206B308A0115
:1028000022206E308A0122206F308A012220773008
:102810008A0122206C308A01222065308A01222020
:1028200064308A01222067308A01222065308A01C3
:10283000222064308A01222020308A0122204F3059
:102840008A0122204B308A01222021308A01222055
:102850000330A300E8308A0158210A308A0122207F
:102860000D308A01222041308A0122206E308A01F7
:10287000222079308A01222020308A0122204B3008
:102880008A01222065308A01222079308A012220A3
:1028900020308A01222054308A0122206F308A01A0
:1028A000222020308A01222045308A0122207830DF
:1028B0008A01222069308A01222074308A01222074
:1028C00021308A0122208A150A1203266400690831
:1028D000053C8A110A160319632C1B308A01222039
:1028E0005F308A01222008000A308A0122200D3040
:1028F0008A01222043308A0122206F308A0122205F
:102900006D308A0122206D308A01222073308A01C5
:10291000222020308A01222045308A012220723074
:102920008A01222072308A0122206F308A012220FF
:1029300072308A01222021308A0122200614831657
:10294000061083120B30A300B8308A0158210610FC
:102950008316061083128A110A162D2C0730B60032
:102960000430B40001308A016F2033308A015720CF
:102970008A016C200730B6000430B40000308A01B0
:102980006F200830A9003C30B000B101A5013830FB
:102990008A01E5208A016C201B308A012220433005
:1029A0008A01222046308A01222061308A012220B9
:1029B0006D308A01222069308A0122206C308A0120
:1029C000222079308A01222020308A0122203D30C5
:1029D0008A01222020308A0122200230A9003808F2
:1029E000A400A5012130B000B1018A01F5206830B2
:1029F0008A0122200A308A0122200D308A012220F9
:102A00000230A9003908A400A5012130B000B101AD
:102A10008A01F5200230A9003A08A400A50121305E
:102A2000B000B1018A01F5200230A9003B08A400E2
:102A3000A5012130B000B1018A01F5200230A900C2
:102A40003C08A400A5012130B000B1018A01F520A5
:102A50000230A9003D08A400A5012130B000B10159
:102A60008A01F5200230A9003E08A400A50121300A
:102A7000B000B1018A01F52068308A0122200A30B5
:102A80008A0122200D308A01222043308A0122202F
:102A900052308A01222043308A01222020308A01CC
:102AA000222056308A01222061308A0122206C3097
:102AB0008A01222020308A0122203D308A012220F2
:102AC00020308A0122200230A9003F08A400A5017D
:102AD0002130B000B1018A01F52068308A0122203E
:062AE0008A110A162D2CDC
:02400E00D423B9
:00000001FF
